:100000000C9446000C9463000C9463000C94630001
:100010000C9463000C9463000C9463000C946300D4
:100020000C9463000C9463000C9463000C946300C4
:100030000C9463000C9463000C9463000C946300B4
:100040000C9463000C9463000C9463000C946300A4
:100050000C9463000C9463000C9463000C94630094
:100060000C9463000C9463000C9463000C94630084
:100070000C9463000C9463000C9463000C94630074
:100080000C9463000C9463000C94630011241FBE55
:10009000CFEFD0E1DEBFCDBF11E0A0E0B1E0E2E202
:1000A000FCE000E00BBF02C007900D92A833B1073F
:1000B000D9F711E0A8E3B1E001C01D92AD33B1075B
:1000C000E1F70C948F050C940000CF93DF93CDB72C
:1000D000DEB722970FB6F894DEBF0FBECDBF9A836E
:1000E000898389819A81009731F089819A8101976A
:1000F0009A838983F6CF22960FB6F894DEBF0FBE9F
:10010000CDBFDF91CF910895CF93DF93CDB7DEB709
:100110008091350084608093350088E795E00E94E7
:1001200065009BEF80913500892380933500DF9136
:10013000CF910895CF93DF93CDB7DEB79EEF809137
:10014000350089238093350080E197E20E946500A5
:1001500080E3809335000E94840088EE93E00E9443
:10016000650080E3809335000E94840088EE93E070
:100170000E94650080E3809335000E94840088EE31
:1001800093E00E94650080E2809335000E94840025
:10019000DF91CF910895CF93DF93CDB7DEB721974D
:1001A0000FB6F894DEBF0FBECDBF898389818F6003
:1001B00080933C0180913500982F906F80913C0195
:1001C0008923809335009EEF8091350089238093A9
:1001D00035000E94840089818295807F80933C0154
:1001E00080913500982F9F7080913C01892B8093DE
:1001F00035009EEF809135008923809335000E9461
:10020000840021960FB6F894DEBF0FBECDBFDF91FC
:10021000CF910895CF93DF93CDB7DEB721970FB677
:10022000F894DEBF0FBECDBF898389818F60809334
:100230003C0180913500982F906F80913C0189237B
:1002400080933500809135008160809335000E9455
:10025000840089818295807F80933C018091350064
:10026000982F9F7080913C01892B8093350080915D
:1002700035008160809335000E94840021960FB67E
:10028000F894DEBF0FBECDBFDF91CF910895CF931D
:10029000DF93CDB7DEB724970FB6F894DEBF0FBE5D
:1002A000CDBF9A8389831C821B8289819A810E9497
:1002B000B7059C018B819C818217930780F42B8169
:1002C0003C8189819A81F901E80FF91F80810E94A0
:1002D0000A018B819C8101969C838B83E6CF2496B7
:1002E0000FB6F894DEBF0FBECDBFDF91CF9108955A
:1002F0000F931F93CF93DF93CDB7DEB7AE970FB6B3
:10030000F894DEBF0FBECDBF69837A838B839C8355
:100310001DA61EA689819A81AB81BC81BB2394F462
:100320008DE20E940A0189819A81AB81BC81B095DE
:10033000A095909581959F4FAF4FBF4F89839A832A
:10034000AB83BC838DA58F5F8DA78DA5282F332709
:10035000C901280F391FCE010196820F931F8C010E
:100360000C5F1F4F89819A81AB81BC812AE030E00C
:1003700040E050E0BC01CD010E94D405DC01CB017E
:10038000F8019183808389819A81AB81BC812AE0C5
:1003900030E040E050E0BC01CD010E94D405DA011C
:1003A000C90189839A83AB83BC8389819A81AB819C
:1003B000BC810097A105B10509F0C4CF8DA58EA71A
:1003C0008EA58DA78DA58823A1F08DA5282F332775
:1003D000C901280F391FCE010196820F931FFC011E
:1003E00034968081805D0E940A018DA581508DA781
:1003F000E9CFAE960FB6F894DEBF0FBECDBFDF914A
:10040000CF911F910F910895CF93DF93CDB7DEB7B2
:100410008AE090E0909339018093380184EF91E075
:1004200090933B0180933A01DF91CF910895CF9350
:10043000DF93CDB7DEB710923B0080E480933A00A3
:1004400010923800109237001092350087EF809399
:10045000340080EC8093320088E080933100109269
:10046000230080E3809322001092620010926100CA
:100470001092650010926400DF91CF910895CF93A0
:10048000DF93CDB7DEB722970FB6F894DEBF0FBE6D
:10049000CDBF80910201909103019A838983898164
:1004A0009A818130910531F089819A81823091055C
:1004B00019F149C084E091E00E94470180EC0E945C
:1004C000CB0085E191E00E9447012091020130912B
:1004D0000301C901820F931FFC01EA5CFE4F80817A
:1004E0009181AA27BB27BC01CD010E9478018DE133
:1004F00091E00E94470127C080E291E00E944701FD
:1005000080EC0E94CB0081E391E00E9447012091A2
:10051000020130910301C901820F931FFC01EA5CC3
:10052000FE4F8081918124E630E0B9010E94C00530
:10053000CB01AA27BB27BC01CD010E9478018DE128
:1005400091E00E94470180E80E94CB0022960FB6FE
:10055000F894DEBF0FBECDBFDF91CF910895CF934A
:10056000DF93CDB7DEB780913900282F332781E0A4
:1005700090E0282739278091000190910101822382
:100580009323817090700097C1F080910201909147
:1005900003018130910539F482E090E090930301EA
:1005A0008093020106C081E090E090930301809364
:1005B00002011092010110920001809139009927E7
:1005C0009C013695279581E090E028273927809176
:1005D0000001909101018223932381709070009714
:1005E000C1F180910201909103018130910551F494
:1005F000809138019091390101979093390180934E
:1006000038010AC080913A0190913B018456904094
:1006100090933B0180933A01809138019091390188
:10062000009731F481E090E0909339018093380194
:1006300080913A0190913B018436910530F484E633
:1006400090E090933B0180933A0110920101109247
:1006500000018091390099279C01369527953695A0
:1006600027953695279581E090E0282739278091B6
:100670000001909101018223932381709070009773
:10068000D1F180910201909103018130910551F4E3
:1006900080913801909139010196909339018093AE
:1006A00038010AC080913A0190913B018C599F4FCB
:1006B00090933B0180933A018091380190913901E8
:1006C0008531910530F084E190E090933901809379
:1006D000380180913A0190913B012BE0893B9207D0
:1006E00030F088EB9BE090933B0180933A011092AD
:1006F0000101109200018091390099279C013295E7
:1007000022952F7023273F70232781E090E0282730
:1007100039278091000190910101822393238170F8
:1007200090700097C1F08091020190910301813097
:10073000910539F482E090E09093030180930201E7
:1007400006C081E090E09093030180930201109233
:100750000101109200018091390099279C012170BC
:10076000307080913900992782709070282B392B36
:1007700080913900992788709070282B392B8091AF
:100780003900992780719070822B932B8B319105C2
:1007900031F481E090E09093010180930001DF91BA
:1007A000CF910895CF93DF93CDB7DEB72E970FB6D5
:1007B000F894DEBF0FBECDBF8091390099279C0110
:1007C000369527953695279581E090E082279327E7
:1007D000817090709C838B831E821D8280910201A8
:1007E000909103018230910521F421E030E03E83B5
:1007F0002D838B819C812D813E81822393230097C1
:1008000009F47EC00E94AF028091390099279C01B3
:10081000369527953695279581E090E08227932796
:100820008170907098878F831A8619868091020153
:10083000909103018230910521F481E090E09A8744
:1008400089878F81988529853A858223932300970C
:1008500039F09FED809123008923806180932300EC
:1008600080913A0190913B019A83898389819A8191
:10087000009731F089819A8101979A838983F6CF15
:100880000E94AF028091390099279C0136952795E7
:100890003695279581E090E08227932781709070AC
:1008A0009C878B871E861D86809102019091030193
:1008B0008230910521F481E090E09E878D878B85C1
:1008C0009C852D853E8582239323009741F080915E
:1008D0002300982F90628FEE8923809323008091CC
:1008E0003A0190913B019A83898389819A8100978B
:1008F00009F462CF89819A8101979A838983F5CF20
:100900002E960FB6F894DEBF0FBECDBFDF91CF910C
:100910000895CF93DF93CDB7DEB766970FB6F894FF
:10092000DEBF0FBECDBF8091390099279C0136955F
:1009300027953695279581E090E08227932781704F
:1009400090709C838B831E821D8280910201909106
:1009500003018130910521F421E030E03E832D83B5
:100960008B819C812D813E8182239323009709F402
:10097000CDC00E94AF020E943F02809139009927AA
:100980009C01369527953695279581E090E0822742
:1009900093278170907098878F831A86198680912B
:1009A0000201909103018130910521F481E090E0F2
:1009B0009A8789878F81988529853A858223932311
:1009C000009731F08FEB90913B00892380933B009F
:1009D0008091390099279C01369527953695279562
:1009E00081E090E082279327817090709C878B87AD
:1009F0001E861D8680910201909103018130910530
:100A000021F481E090E09E878D878B859C852D85E4
:100A10003E85822393230097A1F080913801909125
:100A200039019A83898389819A81009751F00E94C4
:100A3000AF020E943F0289819A8101979A8389833C
:100A4000F2CF8091390099279C01369527953695EC
:100A5000279581E090E08227932781709070988B92
:100A60008F871A8A198A809102019091030181303F
:100A7000910521F481E090E09A8B898B8F8598898C
:100A800029893A8982239323009729F080913B009A
:100A9000806480933B008091390099279C013695B2
:100AA00027953695279581E090E0822793278170DE
:100AB00090709C8B8B8B1E8A1D8A80910201909175
:100AC00003018130910521F481E090E09E8B8D8BB4
:100AD0008B899C892D893E8982239323009709F471
:100AE00022CF80913801909139019A83898389813D
:100AF0009A81009709F417CF0E94AF020E943F022B
:100B000089819A8101979A838983F1CF66960FB67E
:100B1000F894DEBF0FBECDBFDF91CF910895CFEF28
:100B2000D0E1DEBFCDBF0E9417020E949A000E9452
:100B300004028CE00E94CB0081E00E94CB000E9466
:100B4000AF020E943F028091390099278470907013
:100B50000097A9F7809102019091030181309105DE
:100B600019F40E948904EBCF0E94D203E8CFFC0164
:100B700001900020E9F7809590958E0F9F1F0895B2
:100B8000AA1BBB1B51E107C0AA1FBB1FA617B707B3
:100B900010F0A61BB70B881F991F5A95A9F78095CF
:100BA0009095BC01CD01089597FB092E05260ED026
:100BB00057FD04D014D00AD0001C38F4509540954D
:100BC000309521953F4F4F4F5F4F0895F6F7909521
:100BD0008095709561957F4F8F4F9F4F0895A1E24B
:100BE0001A2EAA1BBB1BFD010DC0AA1FBB1FEE1FA7
:100BF000FF1FA217B307E407F50720F0A21BB30BF2
:100C0000E40BF50B661F771F881F991F1A9469F76D
:100C100060957095809590959B01AC01BD01CF01C9
:020C2000089535
:100C220001000200424C494E4B3A20312D32302015
:100C3200202020200053504545443A200020200027
:100C420042555A5A45523A20312D33302020202025
:080C52000054554E453A200004
:00000001FF
